:100000000C94CB030C94E8030C94E8030C94E803E1
:100010000C94E8030C94E8030C94E8030C94E803B4
:100020000C94E8030C94E8030C940C130C9429171B
:100030000C9445280C94E8030C94E8030C94E80312
:100040000C94E8030C94E8030C94E8030C94E80384
:100050000C94E8030C94E3130C94E8030C94E80369
:100060000C94E8030C94E8030C94E8030C94E80364
:100070000C94E8030C94E8030C94E8030C94E80354
:100080000C94E8030C94E8030C94E8030C94E80344
:100090000C94E8030C94E8030C94E8030C94E80334
:1000A0000C94E8030C94E8030C94E8030501098020
:1000B000A101850319012AB700150126B700950192
:1000C00075108100C0050C0901A101850419012AE0
:1000D000A002150126A002950175108100C005013E
:1000E0000906A1018505050719E029E71500250185
:1000F0009508750181020507190029EF15002501F2
:1001000095F075018102050819012905950575010C
:100110009102950175039101C005010902A1010930
:1001200001A100050919012905150025019505758D
:10013000018102950175038101050109300931151D
:1001400081257F95027508810609381581257F95DF
:100150000175088106050C0A38021581257F950175
:1001600075088106C0C005010906A101050719E04F
:1001700029E715002501950875018102950175088B
:1001800081010507190029FF150026FF0095067556
:100190000881000508190129059505750191029549
:1001A0000175039101C0000101010101010101017B
:1001B0000202020202020202020303030303030318
:1001C00003040404040404040505050505060606E5
:1001D0000606070707070708080808090909090AA2
:1001E0000A0A0B0B0B0C0C0C0D0D0D0E0E0E0F0F47
:1001F0000F101011111112121313141415151616D5
:100200001717181819191A1A1B1B1C1D1D1E1E1F43
:100210002020212222232424252626272829292A92
:100220002B2C2D2D2E2F30313232333435363738BA
:10023000393A3B3C3D3E3F404142434445464748B6
:10024000494A4C4D4E4F50515354555658595A5B8C
:100250005D5E5F616264656668696B6C6D6F70722C
:10026000737577787A7B7D7E8082838587888A8C98
:100270008E8F91939596989A9C9EA0A2A3A5A7A9CC
:10028000ABADAFB1B3B5B7BABCBEC0C2C4C6C9CBC3
:10029000CDCFD1D4D6D8DBDDDFE2E4E7E9EBEEF079
:1002A000F3F5F8FAFDFFFFAA7F5540222325262803
:1002B000292A2C2D2F3032333536383A3B3D3E40FB
:1002C00042434547494A4C4E5051535557595A5C41
:1002D0005E6062646668696B6D6F71737577797B58
:1002E0007D7F81838587898A8C8E90929496989A57
:1002F0009C9E9FA1A3A5A7A8AAACAEAFB1B3B4B66C
:10030000B8B9BBBCBEBFC1C2C3C5C6C7C9CACBCCC6
:10031000CDCED0D1D2D2D3D4D5D6D7D7D8D9D9DA99
:10032000DADBDBDBDCDCDCDCDCDDDDDDDDDCDCDC0E
:10033000DCDCDBDBDBDADAD9D9D8D7D7D6D5D4D336
:10034000D2D2D1D0CECDCCCBCAC9C7C6C5C3C2C10B
:10035000BFBEBCBBB9B8B6B4B3B1AFAEACAAA8A768
:10036000A5A3A19F9E9C9A98969492908E8C8A8920
:10037000878583817F7D7B79777573716F6D6B69FD
:1003800068666462605E5C5A5957555351504E4CD2
:100390004A4947454342403E3D3B3A383635333281
:1003A000302F2D2C2A2928262523222E004C002AE6
:1003B00000E100350000001E00140004001D61E093
:1003C000044D001F001A0016001B00E1042A002043
:1003D0000008000700060050002C0021001500094D
:1003E0000019004F004A00220017000A0005000013
:1003F000006564500001580000000F0000E3004F4A
:10040000000258000000070000E20023001C000B5F
:1004100000110000002961240018000D0010005296
:10042000004B0025000C000E00360051002800266D
:100430000012000F0037002F002B0027001300339D
:1004400000387130004E002D0031003400E5001DF1
:100450000100002900010001000100010000003A34
:10046000001E02200222022E002F5D3B001F0221EF
:100470000223020100CA5C3C002F0226022F000169
:1004800000CB5C3D0030022702300001002E5D3EB3
:10049000003102350035020000C45C01000100009B
:1004A00000010000002D5D010001000000010000BE
:1004B00000C35C3F0052005100240200002C5D404C
:1004C00000240021001E000100C85C41002500221C
:1004D000001F003700C65C420026002300200027D2
:1004E00000C75C430025022E0231002E00C95C4487
:1004F00000450001000100010000000100010001B1
:1005000000010001000000010001000100010009DC
:100510005D010001000100F2000100010001000185
:1005200000F000F1000100F400010001000100F3FF
:10053000000100F5000100010001000100010000C0
:1005400000010001000100000001000000010001A5
:100550000001000000010000000100010001000195
:10056000000100000001000100010001000100A9DC
:10057000000100010001000100AC00AA00B600016A
:100580000001000100AB00A8000100010001000112
:1005900000010001000100005C0100AE000100014B
:1005A00000000032190A00047F3F1F6432146432D5
:1005B00014783C1E1E140A050A0000000000030601
:1005C000B200080001000000A800080002000300BB
:1005D000A0001400030057494E555342000000008C
:1005E0000000000000008400040007002A0044000E
:1005F0006500760069006300650049006E007400C4
:1006000065007200660061006300650047005500E8
:10061000490044007300000050007B003900440092
:100620004200370046003100460044002D003700EC
:100630004500370041002D00340030003000380004
:100640002D0039003300360042002D0036004200F4
:1006500041003600430031003900410033003000D2
:10066000380063007D00000000001B0301636F6E13
:100670006669677572652E6572676F646F782D6540
:100680007A2E636F6D0009026B00040100A0FA0965
:1006900004000001030101000921110100012240B1
:1006A000000705810308000A090401000103010293
:1006B00000092111010001224D00070582030800F5
:1006C0000A090402000103000000092111010001D0
:1006D000226D000705830320000A0904030002FFBE
:1006E00000000007058403400005070505034000DE
:1006F000051201100200000008973275490100013F
:1007000002000122034500720067006F0044006F81
:10071000007800200045005A00200053006800695E
:10072000006E006500000030035A005300410020B5
:100730000054006500630068006E006F006C006F7D
:10074000006700790020004C006100620073002007
:100750000049006E006300000004030904050F391E
:1007600000021C100500DF60DDD88945C74C9CD213
:10077000659D9E648A9F00000306B2004500181024
:10078000050038B60834A909A0478BFDA076881566
:10079000B6650001420011241FBECFEFDAE0DEBFD4
:1007A000CDBF23E0ACE9B1E001C01D92A236B20793
:1007B000E1F711E0A0E0B1E0E8EFF7E502C0059055
:1007C0000D92AC39B107D9F70E94BA230C94BB2B18
:1007D0000C940000E8EDF0E080818E7F8083109221
:1007E000E2001092DA001092E100A0EEB0E08C91ED
:1007F00081608C9380818F77808319BCA7EDB0E0F6
:100800008C918E7F8C9380818F7E808310922C03BD
:1008100008952091E4003091E50095E6A90120912A
:10082000EC00822F817020FF06C08091E80080FFDD
:1008300006C080E008952091E80022FD1AC0809152
:100840005103882389F0853089F08091EB0085FD84
:100850000FC02091E4003091E50042175307F9F2F0
:100860009150E1F684E0089582E0089583E00895D0
:1008700081E00895EF92FF920F931F93CF937C0135
:100880008B010E940904C82F882371F08C2FCF910F
:100890001F910F91FF90EF900895F70181917F01D3
:1008A0008093F100015011090115110579F3809130
:1008B000E80085FDF2CF8091E8008E778093E80014
:1008C0000E940904882381F3C82FE0CF809153034D
:1008D00087FF13C08091E80082FF06C08091E80086
:1008E0008B778093E80004C0809151038111F2CF8F
:1008F0000895809151038823D9F38091E80080FF07
:10090000F8CF8091E8008E77ECCF982F9093E90094
:10091000242F762F50E0891731F07091EC00209150
:10092000ED005091F00021FD07C09F5F973071F7F7
:100930008093E90081E008953091EB003E7F309391
:10094000EB003091ED003D7F3093ED003091EB00F6
:1009500031603093EB007093EC002093ED005093E6
:10096000F0002091EE0027FDE0CF80E00895CF92C7
:10097000DF92EF92FF920F931F93CF93DF93C8ED17
:10098000D0E088818F7E8883E7EDF0E08081816010
:10099000808384E082BF81E080932C0388818E7FF6
:1009A000888302EE10E0F80110821092DA0081EEE6
:1009B000C82ED12CF601108288818F778883888198
:1009C0008068888388818F7D888319BC1092510349
:1009D000109252031092500310924F0390EEE92EA2
:1009E000F12CF70180818B7F8083888181608883EF
:1009F00042E060E080E00E948504F60180818E7F05
:100A00008083F80180818160808380818860808319
:100A1000F70180818E7F8083888180618883DF9168
:100A2000CF911F910F91FF90EF90DF90CF9008959D
:100A3000FC018091590390915A0386179707A0F003
:100A40006115710529F48091E8008E778093E800A4
:100A500090E06115710551F4911108C08091E80092
:100A600082FF35C080E00895BC01F2CF8091510330
:100A70008823C9F18530C9F18091E80083FD31C038
:100A80008091E80082FDEACF8091E80080FFE1CF0D
:100A90008091F3002091F200382F6115710519F053
:100AA0002830310558F091E02830310509F090E008
:100AB0008091E8008E778093E800CBCF849180937B
:100AC000F1003196615071092F5F3F4FE6CF809161
:100AD0005103882341F0853041F08091E80083FF85
:100AE000BDCF81E0089582E0089583E00895FC0180
:100AF0008091590390915A0386179707A0F06115CA
:100B0000710529F49091E8009E779093E80090E0B9
:100B10006115710551F4911108C08091E80082FFC0
:100B200034C080E00895BC01F2CF80915103882346
:100B3000C1F18530C1F18091E80083FD30C0809122
:100B4000E80082FDEACF8091E80080FFE1CF80914C
:100B5000F3002091F200382F6115710519F028304B
:100B6000310558F091E02830310509F090E02091EE
:100B7000E8002E772093E800CBCF81918093F1009D
:100B8000615071092F5F3F4FE7CF80915103882358
:100B900041F0853041F08091E80083FFBECF81E0D5
:100BA000089582E0089583E00895089580912E03CA
:100BB000089520915103243091F42093E90070E0CE
:100BC00050E040E00E943A04882321F010922A036A
:100BD00010922B038091E8008E778093E8000895AF
:100BE00090911103803F59F48091120387FF0DC04B
:100BF0001092120391110BC010920D0308C0813F97
:100C000081F48091120318169CF3992381F080914E
:100C1000130390911403892B09F064C010920A0306
:100C20000895823F49F497FFF0CF1092110380910D
:100C300012038111ECCFE0CF833F19F41916ACF306
:100C4000E4CF20911303893F29F41216F4F6109291
:100C50001303DBCF8A3F19F427FFD7CFF8CF2091BA
:100C600014038B3F29F427FFD0CF10921403CDCF6C
:100C70008C3F19F41216CCF3C8CF843F31F4809125
:100C800010038E7F80931003C0CF853F21F48091A5
:100C900010038D7FF7CF863F21F4809110038B7F67
:100CA000F1CF873F21F480911003877FEBCF883FFE
:100CB00021F4809110038F7EE5CF8D3F31F4809138
:100CC000D2028E7F8093D202A0CF8E3F21F48091FA
:100CD000D2028D7FF7CF8F3F09F097CF8091D2025C
:100CE0008B7FF0CF08958091D20280FD1AC081FDE4
:100CF00014C082FD14C080910A03882391F08C33C4
:100D000070F427E0829FC00111246CE370E00E9420
:100D10005329862F672B29F0089583E0089587E0F3
:100D2000089581E008958091D20280FD16C081FD72
:100D300016C082FD18C080910D03882391F08C337A
:100D400090F423E2829FC00111246CE370E00E94C2
:100D50005329862F672B49F0089588E0089581E193
:100D6000089585E0089583E2089581E00895803F25
:100D700031F40E9493068195809312030895813F78
:100D800019F40E949306F8CF823F31F40E94930633
:100D90008195809311030895833F19F40E9493066F
:100DA000F8CF893F29F40E947306809313030895B6
:100DB0008A3F21F40E9473068195F7CF8B3F31F46F
:100DC0000E94730681958093140308958C3F19F453
:100DD0000E947306F8CF843F31F480911003816044
:100DE000809310030895853F21F480911003826061
:100DF000F7CF863F21F4809110038460F1CF873FC5
:100E000021F4809110038860EBCF883F21F480911A
:100E100010038061E5CF8D3F31F48091D202816073
:100E20008093D20208958E3F21F48091D202826095
:100E3000F7CF8F3FB9F78091D2028460F1CF9C0148
:100E40004FB7F8948091CE029091CF02A091D0023A
:100E5000B091D1024FBF821B930B089520912401C2
:100E60002223C9F02091E70227FF15C0E62FE6955F
:100E7000E695E695EE31D8F4E80FF92FF11D67708D
:100E800021E030E001C0220F6A95EAF720958281C7
:100E9000282322830895FC0132960896219162133B
:100EA00003C0DF0111971C92E817F907B9F70895FD
:100EB000209124012223C1F02091E70227FF14C0D2
:100EC000E62FE695E695E695EE31F8F4E80FF92F72
:100ED000F11D677021E030E001C0220F6A95EAF74A
:100EE0008281822B82830895FC0132962FEF30E0BD
:100EF0004191641751F02F3F19F4411101C0232F84
:100F00003F5F3630A9F72F3F09F40895820F911DF6
:100F100027FD9A95FC0162830895CF92DF92EF92AC
:100F2000FF926C01EE24FF2420E0C114D104E104FF
:100F3000F10419F0C701B60120E1C72ED82EE92E21
:100F4000FF24C114D104E104F10419F0285FC701A2
:100F5000B6016B017C0154E0F694E794D794C794F2
:100F60005A95D1F7C114D104E104F10419F02C5FB2
:100F7000C701B6016B017C0142E0F694E794D79477
:100F8000C7944A95D1F7C114D104E104F10419F0D2
:100F90002E5FC701B6019695879577956795672B64
:100FA000682B692B09F02F5F822FFF90EF90DF9065
:100FB000CF9008958091C90281111092C9020895BD
:100FC0008091C8029091C702892B9091C602892B0B
:100FD00080939C019091C9029923A1F0892B809361
:100FE0009C0180912401882341F18091E70287FFD1
:100FF00024C08EE1EEE9F1E090E0815000F591111E
:101000000E94DA07E091EA02F091EB023097E1F0FA
:1010100080912401882359F08091E70287FF07C05F
:1010200080919C0180939D0185E080939C010280CA
:10103000F381E02D8CE991E0099486E0DBCF2191EA
:101040002223D9F29F5FD9CF0895E92FEE0FE90F40
:10105000EE0F8E0F982F977086958695869525E0D2
:10106000829FF0011124E257FD4F50E040E080E004
:10107000219130E0092E02C0369527950A94E2F7B7
:1010800021703327042E01C0220F0A94EAF7822B25
:101090004F5F5F4F4530510559F70895E92FEE0F27
:1010A000E90FEE0F8E0F982F977041E001C0440FAB
:1010B0009A95EAF786958695869595E0899FF00141
:1010C0001124E257FD4F30E020E070E05191DF0144
:1010D0001197CB01022E02C0969587950A94E2F7EC
:1010E000817081958527842385278C932F5F3F4FBF
:1010F0002530310559F7089580918D0290915C0259
:10110000981301C008958F5F8770FACF882341F04C
:1011100080959091C80289238093C8020C94E007BF
:101120000895882339F09091C802982B9093C802B3
:101130000C94E00708952091520230915302281731
:10114000390771F09093530280935202E091EA02C2
:10115000F091EB02309721F00084F185E02D0994A5
:10116000089520915002309151022817390771F0EB
:101170009093510280935002E091EA02F091EB02C9
:10118000309721F00680F781E02D09940895E091D1
:10119000EA02F091EB02309721F00190F081E02D0E
:1011A000099480E00895FA01811101C0FB010994BE
:1011B00080910303982F9E7F29F481708260809331
:1011C000030308958635E8F381708465F8CFAF9204
:1011D000BF92DF92EF92FF920F931F93CF93DF9313
:1011E000082F162FE901E42FF0E0EA55FE4F6111B8
:1011F00011C0E4915E2F4E2F4983E8835A831B82EE
:10120000DF91CF911F910F91FF90EF90DF90BF90F2
:10121000AF900895E62EF12C4491D42EE42FF0E007
:1012200026E0829FC00111242FEF30E0B9010E9417
:101230003F29802F90E0880F991F55E5569FD001D8
:10124000579FB00D11248A1B9B0B982F990F890F64
:101250005901AE18BF08AE9ED001AF9EB00DBE9E24
:10126000B00D11245B2F189F80011124012F11272D
:101270005901A01AB10AAE9E8001AF9E100DBE9E0C
:10128000100D11245901A81AB108AE9CC001AF9CE1
:10129000900DBE9C900D1124892F9927281B390B86
:1012A0002E9FC0012F9F900D3E9F900D1124E92F7E
:1012B00062307105A1F050F46115710509F49CCFFD
:1012C0006130710581F0EB2F512F96CF643071059D
:1012D00069F080F06630710509F48ECFF4CFE42F09
:1012E0004B2F592F89CFE42F412F86CFEB2F542F2F
:1012F000492F82CF4B2F5D2DE12F7ECF9091E702BA
:1013000092FF06C0282F28712830F9F4877F846067
:1013100093FF06C0282F28712831F1F4877E84615D
:101320002091E80220FF06C0382F38713830D9F4F8
:10133000877F816021FF06C0282F28712831D1F4D2
:10134000877E816194FD877E0895282F2471243043
:10135000F9F68B7F8860DCCF282F2471243101F7C8
:101360008B7E8861DDCF382F3171313019F78E7F58
:101370008860E0CF282F2171213121F78E7E88618E
:10138000E1CFCF93DF93972F70E026E0929F600D1F
:10139000711D1124FB0134E5839FE00DF11D112423
:1013A000EE0FFF1FE555FC4FC591D491CE01C23819
:1013B000D105B9F1E8F5C133D10509F499C050F56B
:1013C000C932D10509F48DC0CA32D10509F497C0DC
:1013D000C11521E5D20708F0BFC0C11530E5D3071C
:1013E00008F016C1C83ED10508F09DC0C03ED10529
:1013F00068F5C83AD10508F089C0C53AD10508F0AA
:10140000FFC0C130D10511F1209709F443C02497E2
:10141000E8F440C0C533D10509F45CC0C933D10537
:10142000B9F62091E702237089F080EE90E00EC0BB
:10143000C33ED10591F168F4C03ED105F9F0C23E3A
:10144000D10531F62091E70222FD20C0DF91CF9136
:101450000895C63ED10561F1C73ED10581F1C43E74
:10146000D10509F0B5CF2091E80221FFEFCF80919F
:10147000E70284FD0FC087EE90E0E8CF2091E702FD
:1014800020FD12C13091E80230FFE0CF83EE90E002
:1014900024FFDCCF90E080E0D9CF2091E70222FD4D
:1014A00006C13091E80230FDC0CF24FFCFCFF2CF8C
:1014B0002091E70223FFCACF24FDECCFDCCF20919F
:1014C000E70223FDF7C03091E80231FFEECF84EE52
:1014D00090E0BCCF2091E70225FFB8CF89E290E0F1
:1014E000B5CF2091E70225FFB1CF85E390E0AECFE5
:1014F0002091E70226FFAACF8AE290E0A7CF2091B1
:10150000E70226FFA3CF81E390E0A0CFCF3BD10538
:1015100008F6C85AD0E0CC0FDD1FC15ADE4F8881D3
:101520009981946493CFC11520E2D20760F4C1156C
:1015300031E0D30708F08ACFCE019065C03FD105D6
:1015400008F084CFA7CFC11580E4D80708F4A2CF54
:10155000CE019F70906A7ACFC11595E5D90710F535
:10156000C11524E5D20708F088C0C11533E5D307BB
:1015700008F06FC0C11582E5D80708F465C09E0168
:101580002370332781E090E002C0880F991F2A95CD
:10159000E2F7C695C69520E2C29FE00111248C2B8C
:1015A0009D2B50C0C11599E5D907A0F4C11528E5B8
:1015B000D20708F067C0C11536E5D30708F06ACF37
:1015C0008C2F0E947E0990E0982F882788279F7192
:1015D00090623CCFC1158AE5D80708F458C0CE0107
:1015E00090568115904208F055CF8D2F8F710E9433
:1015F0007E0990E0982F882788279F718C2BE8CF51
:10160000C55AD0E0C45ADE4F888190E090641ECF66
:101610009E01E4E036952795EA95E1F723708C2F3B
:1016200086958695837030E2839FC0011124922BAA
:10163000C37021E030E002C0220F331FCA95E2F7E9
:10164000822B932B9C6802CF9C2F8827816F906AF6
:10165000FDCE9E012370332781E090E002C0880F09
:10166000991F2A95E2F7C695C69530E2C39FE0011F
:1016700011248C2B9D2B9A68E9CE9C2F8827846F90
:10168000906AE4CE9C2F8827806F906ADFCE8C2FE3
:101690008F700E947E0934E0D695C7953A95E1F7A0
:1016A000CF709C2F9069D2CE89E390E0CFCE82EEAE
:1016B00090E0CCCE86EE90E0C9CEBF92CF92DF9282
:1016C000EF92FF920F931F93CF93DF938C01C09003
:1016D0002503D0902603E0902703F0902803809103
:1016E000CA029091CB02A091CC02B091CD02C82A3F
:1016F000D92AEA2AFB2ACFE1D0E0BC2ED701C601C5
:101700000C2E04C0B695A795979587950A94D2F7A5
:1017100080FD0EC0219788F7B12C8B2DDF91CF91E2
:101720001F910F91FF90EF90DF90CF90BF900895A1
:10173000B8018C2F0E94C109019761F3EECFCF93BE
:10174000DF93EC010E945D0BBE01DF91CF910C9401
:10175000C1090E949F0B292F2F7092959F70925064
:101760009E3078F4E92FF0E0E354F44D0C946729AF
:10177000803F19F020F4883E20F481E00895843FF2
:10178000E1F380E00895883EC0F3813FD1F7F5CFC3
:10179000822F869586958695089527982F98089587
:1017A00026982E98089525982D98089556985E9815
:1017B0000895279A2F9A0895269A2E9A0895259A81
:1017C0002D9A0895209828982198299822982A9847
:1017D00023982B9852985A9853985B983E9846981D
:1017E00008958098889A8198899A84988C9A859887
:1017F0008D9A86988E9A87988F9A0895CF93DF93C3
:1018000000D00F92CDB7DEB790915103943019F507
:1018100089837B836A8383E08093E9008FEF9091D3
:10182000E800815095FD06C095ED9A95F1F700000E
:101830008111F5CF8091E80085FF0DC050E040E0B8
:1018400063E070E0CE0101960E943A048091E800C6
:101850008E778093E8000F900F900F90DF91CF91DB
:101860000895BC0184E00C94FE0BBC0183E00C9451
:10187000FE0B9C0182E08093E9009FEF8091E800DD
:10188000915085FD06C085ED8A95F1F70000911114
:10189000F5CF8091E80085FF0CC050E040E065E0A6
:1018A00070E0C9010E943A048091E8008E7780932D
:1018B000E8000895CF93DF93EC0180912401882301
:1018C000B1F18091E70287FF32C060E283E080934C
:1018D000E9008FEF9091E800815095FD06C095EDED
:1018E0009A95F1F700008111F5CF8091E80085FF0E
:1018F0001BC08091240170E050E040E0811104C0E1
:1019000050E040E068E070E0CE010E943A0480912F
:10191000E8008E778093E80080E2FE01AFE2B3E05A
:1019200001900D928A95E1F7DF91CF91089568E0DB
:1019300081E0CDCFEF92FF920F931F93CF93DF9370
:101940000E94D60B0E94D30B0E94D00B0E94CD0B9D
:1019500088E8E82EF12C8FEF90E0F70191838083E7
:101960000AE810E0F80191838083CCE8D0E0998305
:1019700088830E94DF0BFFEF20E782E0F1502040D8
:101980008040E1F700C000000E94DC0B9FEFE0E721
:10199000F2E09150E040F040E1F700C000000E940A
:1019A000D90B2FEF80E792E0215080409040E1F783
:1019B00000C000000E94D30BEFEFF0E722E0E150FF
:1019C000F0402040E1F700C000000E94D00B8FEFF4
:1019D00090E7E2E081509040E040E1F700C0000075
:1019E0000E94CD0B8091D5028770FFEF8F9FC001C1
:1019F000112495958795959587959927F70191835A
:101A00008083F80191838083998388830E94D60B19
:101A10000E94D30B0E94D00BDF91CF911F910F91A9
:101A2000FF90EF900C94CD0BCF9384E090E00E9458
:101A3000102BC82F81E290E00E94102B982F8C2F42
:101A4000CF910895CF92DF92EF92FF926B017C01CC
:101A50000E94D808B701A60188E090E0FF90EF90BF
:101A6000DF90CF900C94362B80910703882319F0D8
:101A70008150809307036091030370910403809168
:101A80000503909106030C94220D80910703833087
:101A900018F48F5F80930703609103037091040330
:101AA00080910503909106030C94220DE3E0F3E08E
:101AB00083E0808311828FEF82838383148260812D
:101AC0007181828193810C94220D6FEE7EEF90E004
:101AD00080E00E94422B60E082E090E00E94242B94
:101AE00060E083E090E00E94242B1092CA021092E2
:101AF000CB021092CC021092CD0260E084E090E024
:101B00000E94242B60E081E290E00E94242B60E0A0
:101B100085E090E00E94242B60E086E090E00E9447
:101B2000242B6FEF87E090E00E94242B40E050E0F0
:101B3000BA0188E090E00E94362B60E08DE090E0F2
:101B40000E94242B40E050E0BA0188E190E00E941E
:101B5000362B60E087E190E00E94242B40E050E0CB
:101B6000BA018CE190E00E94362B60E080E290E0C8
:101B70000E94242B40E050E0BA0188E190E00E94EE
:101B8000362B1092D5021092D6021092D7021092E4
:101B9000D80284E080618093D5024091D5025091B3
:101BA000D6026091D7027091D8028FE090E00E9437
:101BB000362B40E050E0BA0183E190E00C94362BE4
:101BC000CF93C82F873070F580911801909119013B
:101BD000892B89F564E670E080E40E947228909376
:101BE000190180931801892BD1F464E670E082E139
:101BF0000E94CE289093190180931801892B79F4C3
:101C000081E090E001C0880FCA95EAF764E670E0D1
:101C100080950E94CE289093190180931801CF914E
:101C20000C9421298A30B9F040F4883071F0893061
:101C300079F0209A2898CF9108958C3091F070F027
:101C40008D30B9F73E9A4698F6CF219A2998F3CF6E
:101C5000229A2A98F0CF239A2B98EDCF529A5A982D
:101C6000EACF539A5B98E7CFCF93DF93809103033A
:101C700080FD0BC0E9ECF1E0118210821282138228
:101C8000349652E0E530F507B9F7C9ECD1E0FE0132
:101C9000928120813181892F291708F4822F3817EA
:101CA00008F4832F8383381B3183281B2083981BE0
:101CB0009283349682E0E530F80751F70E946C2851
:101CC00064E670E084E80E94722864E670E088812F
:101CD0000E94CE2864E670E089810E94CE2864E6E6
:101CE00070E08A810E94CE2864E670E08B810E94B9
:101CF000CE28249692E0C530D90739F70E942129D1
:101D0000579A3BB13F772BB120684FB7F89489ECD5
:101D100091E0FC015191CF0168E02BB9000000C0B7
:101D200057FF3BB9550F000000C000C000C03BB9D1
:101D300000C06A9591F7F2E085309F0751F74FBFD9
:101D40008FE594E00197F1F700C00000DF91CF919B
:101D500008958F929F92AF92BF92CF92DF92EF92AF
:101D6000FF920F931F93CF93DF93FC01B280948077
:101D700081E08483C5E0D2E009EC11E08BE4A82E79
:101D800088248394EE24EA94F12C2BE4C22ED12CE7
:101D900091101DC01B821A8298014A816981888135
:101DA0000E94E70825960C5F1F4F82E0C035D807D8
:101DB00079F7DF91CF911F910F91FF90EF90DF9016
:101DC000CF90BF90AF909F908F900C94340E2B814A
:101DD000222309F121502B833C818A2D821B311152
:101DE00001C0822F90910603899FC0011124B60182
:101DF0000E943F296A83211104C0332311F01C8201
:101E0000AB8222E02B1540F28091040388838091FD
:101E100005038983C1CF0E94C829823091400CF00C
:101E2000BBCF82E08B15C0F40E94C829B7010E9485
:101E30005329888322E02B1590F40E94C829209111
:101E400005032695622F70E00E945329280F2983ED
:101E50001A82AB828C82A0CF80910403EACF2091BA
:101E60000503F5CFEF92FF921F93CF93DF93EC0121
:101E700089ECE82E81E0F82E10E08C8197014091EA
:101E8000060360910503810F0E94E7081F5E84E04E
:101E9000E80EF11C1F3F89F70E94340E9A818C8155
:101EA00090FF08C08F5F8C83DF91CF911F91FF90CF
:101EB000EF9008958150F7CFBF92CF92DF92EF92CB
:101EC000FF920F931F93CF93DF93FC018281DD2458
:101ED000DA9480FD02C0DD24D39409EC11E0D0E057
:101EE000C0E02FE0B22EF80111821082128213821C
:101EF00094E0E92EF12CC12C8091C6018C0D80312B
:101F00000CF43DC06B2D0E943129892F082E000C46
:101F1000990B8C179D0791F4809106038E9DA0016B
:101F20008F9D500D112455954795559547959801CE
:101F300060910503809104030E94E708CD0CF1E055
:101F4000EF1AF108C9F621960C5F1F4FCF30D1056B
:101F500051F60E94340E8091C60191E0D91215C04D
:101F6000811111C08EE08093C601DF91CF911F9146
:101F70000F91FF90EF90DF90CF90BF90089587FF73
:101F8000C5CF815FC3CF8150EECF90E00196BE01F7
:101F90000E945329E8CF0F931F93CF93DF93C9EC8F
:101FA000D1E0FE011182108212821382349682E007
:101FB000E530F807B9F710E000E08091C701082E7E
:101FC000000C990B081719078CF180911601082E47
:101FD000000C990B801791074CF19E01409106036C
:101FE00060910503809104030E94E7080F5F1F4F73
:101FF00024960F30110509F70E94340E80911501C7
:102000009091C701980F9093C70120911601280F56
:1020100020931601121614F49E301CF081958093C3
:102020001501DF91CF911F910F91089519821882A8
:102030001A821B82DBCF8F929F92AF92BF92CF9278
:10204000DF92EF92FF920F931F93CF93DF93EC01F8
:102050004C81042F10E09801D8010E94AC2B9B0109
:10206000AC010E94772B4B015C01E0E2F0E0E01B49
:10207000F10BA5E5B0E0AC019B010E94772B6B0151
:102080007C019F01DF010E946D299B01AC010E9430
:10209000822B9B01AC01280D391D4A1D5B1DC70118
:1020A000B6010E948A2BF22E822F90E039E23F1572
:1020B000D8F143E0249F9001112435952795122FE4
:1020C000109599ECC92E91E0D92E00E085E5E82E17
:1020D000EF188E2D01FD8F2D9601412F6091050384
:1020E0000E94E7080F5F54E0C50ED11C0F3089F73E
:1020F0000E94340E9C8181E0992319F0903219F4EA
:102100008FEF8093170180911701890F8C83DF91E6
:10211000CF911F910F91FF90EF90DF90CF90BF90E4
:10212000AF909F908F90089525E530E0A901481B5E
:10213000590BCA019A01220F331F280F391F37FF8D
:10214000BCCF2F5F3F4FB9CFEF92FF920F931F93FA
:10215000CF93DF938C01C9ECD1E0F12CE12CF80195
:1021600094816091050380910403F7E0EF16F10478
:10217000FCF49923F9F09E01409106030E94E708C0
:102180002FEFE21AF20A24968FE0E816F10439F7ED
:102190000E94340EF801848190E0019681709927A5
:1021A0008483DF91CF911F910F91FF90EF9008955D
:1021B000992309F39E0140E0E1CF9091030390FF42
:1021C0000DC0E9ECF1E08183608342831382349691
:1021D00092E0E530F907B9F70C94340E08950F93A7
:1021E0001F93CF93DF9300D000D0CDB7DEB78C0123
:1021F0008091C80181110AC09E012F5F3F4F4FEFB0
:102200006FEF0E94E7088A818093C801F80164811A
:10221000613069F08091C80140E0662361F040E0E0
:10222000623011F44091C80180E060E004C0609128
:10223000C80140E080E00E94DD10F801848190E058
:10224000019663E070E00E94532984830F900F9001
:102250000F900F90DF91CF911F910F910895CF9321
:10226000DF9300D000D0CDB7DEB79091030390FF8D
:102270000AC09E012F5F3F4F0E94E7084B81698192
:102280008A810E94DD100F900F900F900F90DF91C8
:10229000CF910895CF93DF93EC01EC81F0E0E55509
:1022A000FD4F4491E3E0F3E0628181810E942F11B0
:1022B0008C818F5F8C83DF91CF910895CF93DF93D3
:1022C000EC01E3E0F3E0438162818C810E942F11F5
:1022D0008C818F5F8C83DF91CF9108955F926F9295
:1022E0007F928F929F92AF92BF92CF92DF92EF92A6
:1022F000FF920F931F93CF93DF9300D000D0CDB701
:10230000DEB7182F762E042F622E9091030390FFD4
:1023100029C0E92FE695AE2FB0E0AF5CBE4F8C919F
:10232000809308039E7F923089F59E012F5F3F4F77
:10233000812F0E94E7084B8169818A810E94DD100C
:10234000109304037092050300930603662051F076
:10235000609103037091040380910503909106033B
:102360000E94220D0F900F900F900F90DF91CF9150
:102370001F910F91FF90EF90DF90CF90BF90AF90A3
:102380009F908F907F906F905F900895823019F4A6
:1023900000910603D5CF863019F410910403D0CFF5
:1023A0008930D9F3893161F6E9518E2F8170582E29
:1023B000E695F0E0EA55FD4FA590B490BB2489EC7A
:1023C000E82E81E0F82ED12CC12C9FE0892E912C93
:1023D000C601B4010E943F29812F511013C0860FFE
:1023E0009701402F672D0E94E708CA0CDB1C84E090
:1023F000E80EF11C85E0E81682E0F80649F70E9435
:10240000340E9ECF861BECCFE3E0F3E043812CE05B
:10241000421B08F440E021E0628181810C946E113E
:10242000E3E0F3E043812CE0420F08F44FEF21E0BA
:10243000628181810C946E11E3E0F3E062812FEF01
:10244000621B08F460E021E0438181810C946E11ED
:10245000E3E0F3E062812FEF620F08F46FEF21E019
:10246000438181810C946E11E3E0F3E0818121E0EE
:10247000438162818C500C946E11E3E0F3E0818122
:1024800021E043816281845F0C946E11E3E0F3E00C
:1024900080818E7F808360817181828193810E949F
:1024A000220D109209032FEF80E792E02150804027
:1024B0009040E1F700C000000C94340E80E290E000
:1024C00090931901809318018091BC0181110EC075
:1024D0000E946C2881E08093BC012FEF83ED90E394
:1024E000215080409040E1F700C0000064E670E0B9
:1024F00080E40E9472289093190180931801892B1F
:1025000009F04EC064E670E080E00E94CE2890930F
:10251000190180931801892B09F042C064E670E02C
:1025200080E00E94CE289093190180931801892B96
:10253000B9F564E670E08FE30E94CE28909319010C
:1025400080931801892B61F50E94212964E670E0CF
:1025500080E40E9472289093190180931801892BBE
:10256000F9F464E670E08CE00E94CE2890931901A3
:1025700080931801892BA1F464E670E080E00E944A
:10258000CE289093190180931801892B49F464E6B1
:1025900070E08FE30E94CE28909319018093180178
:1025A0000E942129809118010895CF93873050F51A
:1025B0008091180190911901C0E0892B71F464E6B3
:1025C00070E081E40E9472289093190180931801B1
:1025D000892B31F0C0E00E9421298C2FCF910895E2
:1025E00084E690E00E94FD2897FF05C090931901B2
:1025F00080931801EFCFC82FC09510921901109247
:102600001801E9CFCFB18FB1869586958C73C370D1
:102610008C2BC82FC095E1CF1F920F920FB60F924F
:1026200011242F933F934F935F936F937F938F93D7
:102630009F93AF93BF93EF93FF938091E10082FF4D
:1026400009C08091E20082FF05C08091E1008B7F8C
:102650008093E1008091DA0080FF24C08091D8004F
:1026600080FF20C08091DA008E7F8093DA00809115
:10267000D90080FF9BC080E189BD82E189BD09B49A
:1026800000FEFDCF81E08093510380912C038111E6
:1026900009C00E94EA030E94B7048091E2008460AE
:1026A0008093E2008091E10080FF17C08091E200FA
:1026B00080FF13C08091E2008E7F8093E2008091C2
:1026C000E20080618093E2008091D8008062809374
:1026D000D80019BC85E0809351038091E10084FF0C
:1026E00029C08091E20084FF25C080E189BD82E19C
:1026F00089BD89B5982F917080FFFBCF8091D8005C
:102700008F7D8093D8008091E1008F7E8093E100DF
:102710008091E2008F7E8093E2008091E2008160F0
:102720008093E20080915203882309F445C084E03D
:10273000809351038091E10083FF27C08091E200E4
:1027400083FF23C08091E100877F8093E10082E0D6
:1027500080935103109252038091E1008E7F809309
:10276000E1008091E2008E7F8093E2008091E200A0
:1027700080618093E20042E060E080E00E94850496
:102780008091F00088608093F000FF91EF91BF91FD
:10279000AF919F918F917F916F915F914F913F91F9
:1027A0002F910F900FBE0F901F90189519BC10928B
:1027B000510310922C0376CF8091E30087FD93E0C4
:1027C00090935103B7CF78941F921FB61F92112494
:1027D0008F939F93AF93BF938091CE029091CF023E
:1027E000A091D002B091D1020196A11DB11D80939C
:1027F000CE029093CF02A093D002B093D102BF91AA
:10280000AF919F918F911F901FBE1F9018952FB76A
:10281000F8948091CE029091CF02A091D002B09115
:10282000D1022FBF08950E9407149C0190911103BB
:1028300080911203982B21F030930F0320930E0305
:102840009091130380911403982B21F030930C0383
:1028500020930B03E091EA02F091EB02309731F004
:102860000480F581E02D80E193E0099408951092B1
:10287000C7021092C6020E94E00785E0E0E1F3E0A3
:10288000DF011D928A95E9F710920D0310920A0359
:102890001092D2020E94131490E080E00E94B108CE
:1028A00090E080E00C949B086093CA027093CB0286
:1028B0008093CC029093CD020C9437141092C802EE
:1028C00080912401EEE9F1E0882359F08091E7023C
:1028D00087FF07C08EE1DF011D928A95E9F70C940E
:1028E000371486E0F8CF1F93CF93DF93CDB7DEB7D1
:1028F000AA970FB6F894DEBF0FBECDBF83E593E075
:102900002091F100FC012193CF01F3E08B359F076B
:10291000B9F780915403893009F444C018F5823026
:1029200009F4B9C0833009F46EC0813031F580916B
:102930005303813A11F58091E800877F8093E80086
:102940008091570390915803892B41F560E28FE203
:1029500093E070E00E9477058091E8008B77809388
:10296000E8000BC08B3009F46BC008F483C08234DC
:1029700009F4A2C0853409F4BCC08091E80083FF4B
:1029800050C280915303909154039A3008F049C289
:10299000E92FF0E0E553F44D0C94672960E090E0F6
:1029A00080E0D7CF80915303813239F7809157036C
:1029B00090915803009711F00297F9F68091E80082
:1029C000877F8093E8008091E80082FF17C0909194
:1029D000F3008091F200029729F48091F1008B7F3F
:1029E000813021F48091F10080932E038091E800E2
:1029F0008B778093E8000E946604BFCF80915103DB
:102A00008111E1CFBACF80915303813A09F0B5CF5C
:102A10008091570390915803892B09F0AECF809194
:102A2000E800877F8093E8008091E80080FFFCCF7A
:102A3000809124018093F1008091E8008E77D9CFB6
:102A400080915303813209F098CF80915703909180
:102A50005803892B09F091CF8091E800877F8093FC
:102A6000E8000E94660480915503809324010E942F
:102A70005E1483CF80915303813209F07ECF809121
:102A8000E800877F8093E8000E94660480915603E7
:102A900080932D0372CF80915303813A09F06DCF5B
:102AA0008091E800877F8093E8008091E80080FFB4
:102AB000FCCF80912D03BECF80915303803C09F061
:102AC0005CCF8091570390915803029739F580911C
:102AD000550390915603892B09F58091E800877F73
:102AE0008093E8006BE170E08AE696E00E941805AA
:102AF00082CF80915303803C09F03FCF80915703F0
:102B000090915803079751F48091E800877F809354
:102B1000E80062EB70E088EB95E0E8CF8091EB0095
:102B200080628093EB0029CF803899F0823809F0D9
:102B300078C1809157038F70873008F072C18093FD
:102B4000E9008091EB0085FB882780F91092E9006D
:102B500006C080914F039091500391118260909133
:102B6000E800977F9093E8008093F1001092F100C5
:102B70008091E8008E7751C1882309F43FC18230EB
:102B800009F04FC180915503811142C180915703D3
:102B90008F702FEF280F263008F043C18093E90093
:102BA0002091EB0020FF34C1933031F48091EB0091
:102BB00080628093EB002CC19091EB009061909328
:102BC000EB0021E030E001C0220F8A95EAF7209364
:102BD000EA001092EA008091EB008860EACF811150
:102BE00020C1109155031F778091E3008078812BDD
:102BF0008093E3008091E800877F8093E8000E9443
:102C000066048091E80080FFFCCF8091E30080683B
:102C10008093E30082E0111183E08093510301C1AE
:102C20008058823008F0FDC0809155039091560382
:102C30008C3D23E09207A1F583E08A838AE28983B1
:102C40004FB7F894DE01139620E03EE051E2E32F07
:102C5000F0E050935700E49120FF03C0E295EF703D
:102C60003F5FEF708E2F90E0EA30C0F0C7968D93F3
:102C70009D932F5F243159F74FBF8091E800877FE4
:102C80008093E8006AE270E0CE0101960E94770529
:102C90008091E8008B778093E800C3C0C096E7CFAF
:102CA0002091570330915803492F55274330510540
:102CB00051F1A0F44130510509F459C06BE670E0C0
:102CC00086E896E04230510509F0ABC02091E8005B
:102CD000277F2093E8000E941805DACF4132510582
:102CE00039F14232510591F14F30510509F099C047
:102CF000EFE5F7E0649170E08DE597E0611571050F
:102D000009F48FC0E3CF99278130910571F00097C6
:102D100031F0029709F085C0E3E0F7E002C0E9E591
:102D2000F7E0649170E0CF01E9CFE7E2F7E0F9CF97
:102D30002330310508F075C0220F331FF901EA5620
:102D4000FE4F8081918169E070E0C0CF2330310572
:102D500008F067C0F901EE0FFF1FE057FE4F8081BA
:102D6000918123573E4FF901608170E0C7CF62E146
:102D700070E081EF96E0AACF803809F052C08091D0
:102D8000E800877F8093E800809152038093F100F0
:102D9000EFCE811146C010915503123008F041C0AA
:102DA0008091E800877F8093E800109352030E948F
:102DB0006604112311F084E005C08091E30087FDD3
:102DC000FACF81E08093510342E061EC81E00E9400
:102DD000850442E061EC82E00E94850442E261ECFD
:102DE00083E00E94850442E361EC84E00E94850454
:102DF00042E360EC85E00E94850413C08091550396
:102E0000813079F481E0933009F080E080935003C1
:102E10001092E9008091E800877F8093E8000E948B
:102E200066048091E80083FF0AC08091E800877FF4
:102E30008093E8008091EB0080628093EB00AA967B
:102E40000FB6F894DEBF0FBECDBFDF91CF911F91BB
:102E500008951F920F920FB60F9211242F933F9354
:102E60004F935F936F937F938F939F93AF93BF9392
:102E7000CF93DF93EF93FF93D091E900DF708091C0
:102E8000EC00C82FC17080FDC0E81092E90080916D
:102E9000F000877F8093F00078940E947314109262
:102EA000E9008091F00088608093F000CD2BCF7016
:102EB000C093E900FF91EF91DF91CF91BF91AF9166
:102EC0009F918F917F916F915F914F913F912F9142
:102ED0000F900FBE0F901F9018958823B1F19CEFB3
:102EE000980F913A38F4682F8CE991E00E942E07F0
:102EF0000C94E00790E2980F983088F4877021E0F6
:102F000030E0A90102C0440F551F8A95E2F7CA01BB
:102F100080959091C80289238093C802E9CF9BE5F0
:102F2000980F933020F490E080E00C94B10898E57D
:102F3000980F973120F490E080E00C949B08803F3C
:102F400020F00E94F0050C9413140895CF93C82F1D
:102F5000882309F46EC08CEF8C0F813AB8F580910C
:102F60002401882311F18091E70287FF1EC0EC2F16
:102F7000E695E695E695F0E0E456FE4F828190E016
:102F80004C2F477021E030E002C0220F331F4A95DA
:102F9000E2F782239323892B89F06C2F8CE991E04F
:102FA0000E942E070E94E00709C0EEE9F1E081913E
:102FB000C81799F381E0E43AF807C9F76C2F8CE958
:102FC00091E00E945807CF910C94E00780E28C0FAB
:102FD000883068F4C77021E030E001C0220FCA9544
:102FE000EAF78091C802822B8093C802ECCFEBE510
:102FF000EC0FE33040F4F0E0E45AFE4F808190E0C3
:10300000CF910C94B108E8E5EC0FE73150F4F0E013
:10301000EE0FFF1FE15AFE4F80819181CF910C94FA
:103020009B08C03F30F08C2F0E94B706CF910C94C4
:103030001314CF9108950F931F93CF93DF93C62F4F
:10304000D42F022FFC0182818823A1F060935D03BD
:103050000E94071490935C0380935B03C77081E028
:1030600001C0880FCA95EAF7DF91CF911F910F91A8
:103070000C94910880915D03681338C080915B03C4
:1030800090915C030E941F078639910578F510E244
:103090001D0FCD17B9F080E28C0F883040F4C77057
:1030A00081E001C0880FCA95EAF70E9486081830AF
:1030B00048F481E09D2F977001C0880F9A95EAF738
:1030C0000E949108802F0E94A617802F0E946D17E2
:1030D000183098F4D77081E001C0880FDA95EAF7CC
:1030E000DF91CF911F910F910C948608C77081E0FA
:1030F00001C0880FCA95EAF7F3CFDF91CF911F91F6
:103100000F91089560910303669570E04BE050E0E5
:103110008AE091E00E94032B892B19F481E08093CF
:1031200009030E9407149093FE028093FD02089504
:103130009091030390FF36C09170811129C0926075
:1031400090930303662351F060910303709104038D
:1031500080910503909106030E94220D6091030364
:10316000669570E04BE050E08AE091E00E94032B0E
:10317000892BA9F01092090381E08093000320E0DD
:103180004091060360910503809104030C946E1135
:103190008B3210F09465D4CF880F982BD1CF0E943A
:1031A0008218EACF0895E3E0F3E0808181608083B4
:1031B00060E086950C94981861E00C949818E3E010
:1031C000F3E080818160808386950C94DC18809187
:1031D00003038695815009F48AE261E00C94981803
:1031E0008091030386958F5F8B3208F081E061E068
:1031F0000C9498189091030390FF07C09695981728
:1032000020F0961710F40C94F0180C94DC18CF9260
:10321000DF92EF92FF92CF93DF936B017C010E94CC
:103220008D07C82F0E94D60B0E94D30B0E94D00B93
:103230000E94CD0BD0915402C150C73090F5EC2FB5
:10324000F0E0EB52F44D0C9467290E94DF0BD11192
:103250000CC00E94D31860E081E00E94981820E022
:103260004FE968EE8CED0E946E11C701B601DF9147
:10327000CF91FF90EF90DF90CF9008950E94DC0BEC
:10328000D111F3CF0E94D31860E081E00E9498181A
:1032900020E04FE96AEF8BE8E6CF0E94DF0B0E9447
:1032A000DC0BD111E2CF88E090E00E94182B6093F4
:1032B000030370930403809305039093060360FF58
:1032C00019C00E94DF188091030386950E94DC18C4
:1032D00021E0409106036091050380910403C3CF70
:1032E0000E94DF0B0E94D90BDCCF0E94DF0B0E94F3
:1032F000DC0BF8CF0E944612B8CFCF92DF92EF924C
:10330000FF92CF93DF9300D000D0CDB7DEB70E94FD
:1033100007196B017C0180912903882321F080919A
:103320002A03811115C0C0922503D0922603E09292
:103330002703F09228030E9437140F900F900F90EC
:103340000F90DF91CF91FF90EF90DF90CF90089595
:10335000198282E08A83C701B6010E948D078B83A0
:103360008EEF8C8364E0CE0101960E94D905DBCFFD
:103370000F931F9341E050E060E070E004C0440F01
:10338000551F661F771F8A95D2F7CB01BA0160954A
:1033900070958095909500912503109126032091BA
:1033A00027033091280360237123822393231F91E5
:1033B0000F910C947D199091C5028095892380937B
:1033C000C502282F277071F4282F082E000C330B0C
:1033D0009217130639F08595859585950E94B81941
:1033E0001092C50208950F931F9341E050E060E0F2
:1033F00070E004C0440F551F661F771F8A95D2F7EF
:103400008091250390912603A0912703B091280372
:103410008A019B01082B192B2A2B3B2BC901B801D0
:103420001F910F910C947D194F925F926F927F9232
:103430008F929F92AF92BF92CF92DF92EF92FF92C4
:103440000F931F93CF93DF9300D000D00F92CDB78F
:10345000DEB77C01FC0183819481892B39F01081D6
:10346000D180812F8D218F3F09F0B7C50F900F902C
:103470000F900F900F90DF91CF911F910F91FF90C0
:10348000EF90DF90CF90BF90AF909F908F907F9004
:103490006F905F904F9008950E945D0B082F682FEA
:1034A00089819A810E944E08E12FF0E026E0D29EA9
:1034B000E00DF11D112434E5039FE00DF11D1124F1
:1034C000EE0FFF1FE555FC4F0591149180912903E4
:1034D000882321F080912A0381116BC50A32FDE512
:1034E0001F0709F08AC0F70182818823C9F1809102
:1034F000D50291E0980F9770887F953008F4892B5A
:103500008093D5028091D5028770FFEF8F9FC00115
:10351000112495958795959587959927909389007E
:103520008093880090938B0080938A0090938D0005
:1035300080938C004091D5025091D6026091D702C1
:103540007091D8028FE090E00E94362B60912503A5
:103550007091260380912703909128030E940719F8
:10356000F7019281992309F449C510925D03023055
:10357000FCE51F0708F4BFC106312CE5120738F03F
:1035800098012B5F3C452730310508F0B4C10E94FB
:10359000140D9093E8028093E7020F303CE5130787
:1035A00009F48AC108F004C108309CE5190709F440
:1035B0006DC108F0D9C00430FCE51F0709F45AC1F9
:1035C00008F0BFC002303CE5130709F44BC10330DB
:1035D0001C4509F44BC16091E7021091E80284E0B8
:1035E00090E00E94242B612F81E290E00E94242B26
:1035F0000E945E1467C081E1E2C40D322DE512071E
:1036000009F46EC018F50B328DE5180709F450C0A7
:103610000C329DE5190709F443C0043F2CE512075D
:1036200009F480C050F5093D8CE5180709F476C00F
:103630000A3D9CE5190709F481C0083DECE51E0729
:1036400009F08ECF26E241EE61EE26C00E32EDE5A6
:103650001E0709F455C00F32FDE51F07F1F6F7010B
:103660008281882379F10E94DF1881E00E94DC18B2
:1036700021E04FEF6FEF8BE140C0063FFCE51F07F5
:1036800009F458C008F452C027E245EE66EE073F41
:103690003CE5130709F064CFC7010E941B1812C054
:1036A000F7018281882371F081E00E94DC180AC052
:1036B000F7018281882331F08091540291E08927BB
:1036C000809354028091C502877009F4CFCEF70130
:1036D0008281882309F4CACE82E00E94DB19C6CE1B
:1036E000F7018281882371F30E94DF1881E00E9434
:1036F000DC1821E04FEF6FEF8CEA0E946E11E2CFF1
:10370000F70182818823F1F20E94DF1881E00E9494
:10371000DC1821E040E86FEF86E5EFCF27E245EEC9
:1037200065EEBACF26E241EE60EEB6CF27E245EE77
:1037300064EEB2CF26E241EE62EEAECF28E241E087
:10374000EFCF8091E702806106309CE5190709F40C
:1037500047C08091E702886007301C4508F440C0EC
:103760008091E70280623CC00B30FCE51F0709F442
:103770009BC068F409303CE5130709F48BC00A309C
:103780001C4509F028CF8091E7028C6029C0809108
:10379000E7028B7F0D309CE5190711F18091E7025C
:1037A0008D7F0E301C45E0F08091E702877F18C0C6
:1037B0000B3FFCE51F0709F461C060F502313CE5F1
:1037C000130709F481C078F400319CE5190709F466
:1037D00077C08091E7028F7B01311C4509F0FBCE59
:1037E0008093E702F8CE0431FCE51F0709F47AC0A4
:1037F00008F470C005311C4509F0EDCE8091E70258
:1038000082FB992790F921E0922790FB82F990FBA7
:1038100083F9E6CF0E3F8CE5180709F449C070F430
:103820000C3FECE51E0771F18091E8028E7F0D3FA1
:103830001C4509F0D0CE8093E802CDCE01152DE5D0
:10384000120709F44BC060F101301D4509F0C3CEE9
:103850008091E802982F909591708E7F892B90FB34
:1038600081F9E9CF8091E7028160BACF8091E702C8
:103870008260B6CF8091E7028460B2CF8091E80287
:103880008160D9CF8091E8028260D5CF8091E70234
:103890008064A6CF0E945E148091E7028068A0CF6A
:1038A0008091E8028360C7CF8091E7028E7F98CF36
:1038B0008091E8028D7FBFCF8091E7028F7E90CF0D
:1038C0008091E7028F7D8CCF0E945E148091E70289
:1038D0008F7786CF8091E702837F82CF8091E80245
:1038E0008C7FA9CF0E945E149091E702892F97FBED
:1038F00087F9805875CF8091C8020631ECE51E0724
:1039000009F08AC38A7A91E009F490E09093550215
:1039100069E2811165E38CE991E00E9458070E94F9
:10392000E007D0CE8091030380FF03C00E944612BF
:10393000C9CE0E94DF18C6CE47EE58E160EF78E1AD
:103940000E94D308BFCE40EF58E167EE78E1F8CF90
:1039500044E352E16DE372E1F3CF4DE352E164E3FE
:1039600072E1EECF4CE152E168E272E1E9CF48E268
:1039700052E16CE172E1E4CF44E052E160E172E1D6
:10398000DFCF40E152E164E072E1DACF44E35DE091
:1039900065E47DE0D5CF45E45DE064E37DE0D0CF34
:1039A00065E082E00E94FA188DCE68E086E0FACFEA
:1039B0006EE089E0F7CF64E18FE0F4CF67E185E165
:1039C000F1CF88E172CE62E289E1ECCF83E26DCE85
:1039D0000F3DFCE51F0709F446C009302DE512072D
:1039E00009F444C001151C4509F047C00E945E144B
:1039F0008FEF94E3ECE081509040E040E1F700C0AD
:103A00000000F89481E08093E00080E28093D80089
:103A10001092C9008FE19EE40197F1F700C0000009
:103A20001DBA109268001CBC10BE1FBA10927A001A
:103A300010926E0010926F0010927100109272003E
:103A40001092C9001092BC0014B817B81AB81DB86B
:103A500010BA1092BC0015B818B81BB81EB811BA2D
:103A60000C94003F2FCE0E94650D2CCE80912B032D
:103A700091E0892780932B0325CEF70100811181E6
:103A8000992309F43DC0C8010E945D0BD82E682F10
:103A9000C8010E944E08B8018D2D0E94C1098C01F9
:103AA000882EF701A580A2944FE0A422D280D110E5
:103AB0001092C7028091C502877099F0DD2089F0CD
:103AC000812F807F803421F080E2800F883048F0A1
:103AD00082E00E94DB198091C5028770CC24C394D8
:103AE0008111C12CB12EB2943FE0B322FBE0FB1553
:103AF00008F440C0EB2DF0E0E452F44D0C9467293B
:103B0000C8010E942508D82EC6CF212F2F70A22EC3
:103B1000107F19F0A29420EFA222DD20C9F0AA2084
:103B200069F080E2800F883010F081100BC0809126
:103B3000C802A82AA092C8020E94E007802F0E9413
:103B4000A61718C08091C702A82AA092C702F4CF76
:103B5000802F0E946D17AA2069F0A094005E0830A3
:103B600010F0811046C08091C802A822A092C8021D
:103B70000E94E0072B2D2850330B2430310510F420
:103B80000E94C708CC20A9F08091C50280FD11C019
:103B9000F70112828595859585950E94F319C701D5
:103BA0000E94141A8091C5028595859585950E947D
:103BB000B81985E0F701DE01119601900D928A9502
:103BC000E1F789819A810E9425089A81E981F0E0D4
:103BD00026E0929FE00DF11D112434E5839FE00D56
:103BE000F11D1124EE0FFF1FE555FC4F85919491B7
:103BF0003DCC8091C702A822A092C702B9CF312F35
:103C00003F70932E107F103219F0929490EF99220A
:103C1000882041F081E0881631F1DD2079F1AA2079
:103C200041F18CCFDD2091F09091C902892D892B33
:103C3000A11003C00E9491089DCFE1E0AE12FACF1F
:103C4000981709F497CF8093C90294CFA11006C0AA
:103C50000E94DA07892D0E9486088CCFF1E0AF160A
:103C600009F488CFF5CFDD2031F021E02A1508F4E2
:103C700081CF892DDFCFA1107DCFECCFAA2051F3CA
:103C800039E383128FC18FEF97EEE3E081509040CC
:103C9000E040E1F700C0000085C1812F8695869540
:103CA000837061F0813009F065CFC8019370D11045
:103CB00002C090E080E00E949B085CCFC801937036
:103CC000D11002C090E080E00E94B10853CF802F55
:103CD000DD2029F00E94B7060E9413144BCF0E94EA
:103CE000F005FACF812F837009F066C0D11042CF62
:103CF000802F829586958770880F880F602F6F7050
:103D0000462E512C712C612C082E04C0440C551CDD
:103D1000661C771C0A94D2F740E050E0BA0104FF19
:103D20000FC04FE050E060E070E004C0440F551F4A
:103D3000661F771F8A95D2F74095509560957095CC
:103D4000812F869586958370823019F1D8F4009181
:103D5000CA021091CB022091CC023091CD02813069
:103D600069F04429552966297729CB01BA016023D6
:103D70007123822393230E945414FCCE402A512A9B
:103D8000622A732ACB01BA016429752986299729E9
:103D9000F2CF44295529662977290091CA0210914A
:103DA000CB022091CC023091CD02CB01BA01602729
:103DB000712782279327DFCF8695DD2011F0812F91
:103DC0008170882309F4D6CE802F829586958770DE
:103DD000880F880F602F6F70462E512C712C612C2C
:103DE000082E04C0440C551C661C771C0A94D2F79C
:103DF00040E050E0BA0104FF0FC04FE050E060E047
:103E000070E004C0440F551F661F771F8A95D2F7D4
:103E10004095509560957095812F86958695837015
:103E2000823019F1D8F400912503109126032091D6
:103E3000270330912803813069F0442955296629E8
:103E40007729CB01BA0160237123822393230E9437
:103E50007D1990CE402A512A622A732ACB01BA01D9
:103E60006429752986299729F2CF4429552966297D
:103E70007729009125031091260320912703309183
